:100000000EC015C014C013C012C011C010C00FC064
:100010000EC00DC00CC00BC00AC009C008C011241E
:100020001FBECFE5D1E0DEBFCDBFA4D0B0C1E8CFC9
:10003000009741F0E9EFF0E03197F1F700C00000E0
:100040000197F6CF089589BD2AB52F77892B11F036
:1000500080E801C080E0282B2ABD0895892B11F487
:10006000CB01F1CF68BD8AB58F7D672B11F090E28F
:1000700001C090E0892B8ABD089581E087B981E0B5
:1000800090E0D6DF369A3699FECF84B125B190E064
:10009000922B0895009769F02AE030E0E7EAF1E654
:1000A0003197F1F700C0000021503109B9F70197ED
:1000B000F1CF0895FC01CA01718360836FEF70E096
:1000C00041D164E670E04FD1778366831582148254
:1000D000138212820895FC0180819181BFCFFC01BF
:1000E000CB01228133812115310529F021503109BD
:1000F0003383228308956536710568F4009769F4A7
:1001000084819581009721F00197958384830895D8
:1001100060E070E023C084E690E020813181232BF1
:1001200011F429B501C028B530E042E350E0558311
:100130004483232B39F48FE090E0938382836FEF25
:1001400070E00CC0268137816FEF70E0621B730B8B
:10015000F9D064E670E007D1620F731FCF01BBCF07
:10016000FC0180819181892B11F489B501C088B58A
:1001700090E00895CF93DF93CDB7DEB760970FB6C9
:10018000F894DEBF0FBECDBF329A319A309A379ABB
:10019000B89AB99A18BC19BC83E08ABD13BE81E035
:1001A00083BF80E090E04FDF60E070E081E090E0AE
:1001B00055DFBA98BB98BC9884E690E039DF8FEFA2
:1001C00090E041DF83E090E065DF80E090E03BDF9E
:1001D00082E390E02DDF6FEF70E081E090E03EDFA2
:1001E00083E090E057DF60E070E081E090E036DF90
:1001F00085E090E04FDF8FEF90E025DF6FEF70E05C
:1002000081E090E02BDF83E090E044DF80E090E04D
:100210001ADF60E070E081E090E020DF85E090E0B0
:1002200039DF2BDF5C011A86198682EB90E0988B10
:100230008F871E861D861C861B8621E030E03A8350
:10024000298398878F831E821D821C821B82512CDA
:10025000CE0101967C018E01075F1F4F43E2342ED1
:1002600052E2452E62E3862E912C07DF6C0137B8EF
:1002700081E090E0DDDE369A3699FECF65B0712CD4
:1002800047B881E090E0D4DE369A3699FECF25B1AA
:10029000C50161E370E056D08C0D9D1DB40163D0A3
:1002A0005B016D3291E0790720F0CB018C529140D7
:1002B00002C080E090E07694679468167906B0F406
:1002C0008619970964E670E03DD0622F70E076955C
:1002D000679549D06B016536710568F03B0194E67E
:1002E000691A710884E6C82ED12C07C0612C712CC4
:1002F000C12CD12C02C0612C712CB601C801EFDEDB
:10030000B301C701ECDE511002C0CD28A9F0C8012D
:1003100027DF892B21F4C70123DF892B19F055240E
:1003200053940AC0512C84E690E082DE902F812FF6
:100330008701E92EF82E99CF9E2D8F2D7801092F58
:10034000182FF1CF0024552704C0080E591F880F1D
:10035000991F009729F076956795B8F37105B9F75D
:10036000802D952F0895AA1BBB1B51E107C0AA1F22
:10037000BB1FA617B70710F0A61BB70B881F991F46
:100380005A95A9F780959095BC01CD010895F894F0
:02039000FFCF9D
:00000001FF
